:100000000C9469000C9491000C9491000C94910054
:100010000C9491000C9491000C9491000C9491001C
:100020000C9491000C9491000C9491000C94DB09B9
:100030000C9491000C9491000C9491000C949100FC
:100040000C9459110C9491000C9459130C948B132B
:100050000C9491000C9491000C9491000C949100DC
:100060000C94BB080C9491000000000900030200EE
:10007000000405080000000000000000000000016E
:10008000020408102040800102040810200102042C
:100090000810204080400404040404040404020204
:1000A000020202020303030303030202030000002F
:1000B0000023002600290000000000250028002B56
:1000C0000000000000240027002A00002003F4079D
:1000D000BB1311241FBECFEFD8E0DEBFCDBF12E0AF
:1000E000A0E0B1E0ECE9FCE202C005900D92A03383
:1000F000B107D9F724E0A0E3B2E001C01D92A63A0F
:10010000B207E1F710E0C9E6D0E004C02197FE0194
:100110000E941716C636D107C9F70E94D7140C944F
:100120004C160C940000862F642F0C94C612FC0110
:1001300081890E94301321E0892B09F420E0822F6D
:100140000895FC01DB0182E791E0918380831296A0
:100150004D915D916D917C9115974283538364839A
:10016000758316968D919C91179797838683189621
:100170008C911897808719964D915D916D917C9126
:100180001C9741875287638774871D964D915D91B7
:100190006D917C915097458756876787708B5196F4
:1001A0008C915197818B88E791E09183808352965F
:1001B0008C91828B0895CF92DF92EF92FF920F93F2
:1001C0001F93CF93DF930E94C60B8BEE92E00E94A9
:1001D00004078BEE92E00E9409068BEE92E00E94EB
:1001E000540601E811E0C3E5D2E085E8C82E81E0BD
:1001F000D82E7801F70161917F0170E0CE010E9455
:10020000DC0565E070E0CE010E9446051A8A63961F
:10021000CE14DF0479F763E070E080E592E00E949D
:10022000300B6091030170E080E592E00E946B0B5F
:1002300080E492E00E94AF0D80E392E00E94AF0D57
:1002400061E084E00E94C61261E08EE00E94C61266
:1002500061E08FE00E94C61261E085E00E94C61254
:1002600061E086E00E94C61261E089E00E94C61249
:1002700060E081E10E94C61260E082E00E94C61246
:1002800062E0F80181918F010E94C612F1E0063808
:100290001F07B1F761E084E00E94021370E060E0A4
:1002A00085E00E94401270E060E086E00E9440120B
:1002B00070E060E089E00E9440128FE580930903BE
:1002C00080930A0380930B0380930C0380930D03A8
:1002D00080930E0380930F0380931003DF91CF91DF
:1002E0001F910F91FF90EF90DF90CF9008950F93A3
:1002F0001F93CF93DF938B01EA01BC0185E00E943D
:100300004012B80186E00E944012BE0189E0DF91F0
:10031000CF911F910F910C94401250E040E070E09B
:1003200060E090E080E00C947701813041F028F0AB
:10033000823069F0833091F008950C948D0150E083
:1003400040E070E060E08FEF90E00C94770150E0C7
:1003500040E06FEF70E090E080E0F7CF4FEF50E0CB
:1003600070E060E0F8CF0E943C1661E0892BA1F5B7
:1003700086E00E9402138BEE92E00E94540640E059
:1003800065E08BEE92E00E94620663E371E08BEE23
:1003900092E00E94241441E062E08BEE92E00E9421
:1003A00062066AE371E08BEE92E00E942414809171
:1003B0000001809301016091020170E080E592E00C
:1003C0000E946B0B60E086E00E94021368E873E114
:1003D00080E090E00C94D41185E00E9402138BEE33
:1003E00092E00E94540640E065E08BEE92E00E94AD
:1003F000620663E371E08BEE92E00E94241441E018
:1004000065E08BEE92E00E94620666E471E08BEE9E
:1004100092E00E94241468EB7BE080E090E00E9470
:10042000D41160E085E00C940213AF92BF92CF929A
:10043000DF92EF92FF920F931F93CF93DF937C0194
:10044000FC0101900020E9F731978F01081B190B7F
:10045000680120E1C21AD10880E1A82EB12C809158
:10046000F70280171106A1F041E060E08BEE92E008
:100470000E94620601311105C4F4B7018BEE92E0CF
:100480000E94241468EB7BE080E090E00E94D4118D
:100490001092F702DF91CF911F910F91FF90EF9093
:1004A000DF90CF90BF90AF9008958091F70290E0D9
:1004B000E701C80FD91F8C159D052CF52091F70277
:1004C000822F90E00F96AE014E195F0984179507B1
:1004D00034F069918BEE92E00E942C14EFCF211141
:1004E00006C06CED75E080E090E00E94D4116CE2F3
:1004F00071E080E090E00E94D4118091F7028F5F5C
:100500008093F702ACCFCE018E199F098017910717
:1005100034F469918BEE92E00E942C14F4CFD0E079
:10052000C0E08091F7029801281B3109C9019501AB
:10053000281B390B2C173D07D4F260E28BEE92E0BA
:100540000E942C142196EDCF1F93CF93DF93CDB74C
:10055000DEB7CC58D1090FB6F894DEBF0FBECDBFC1
:10056000182F8BEE92E00E9454068BEE92E00E94D0
:100570000E0640E060E08BEE92E00E9462066EE4C0
:1005800071E08BEE92E00E9424144AE050E0612F6B
:100590008BEE92E00E948C14123079F108F5609194
:1005A0001C0170911D01113019F1CE0101960E94BC
:1005B00015028BEE92E00E94540680910101843076
:1005C00020F48BEE92E00E940906C457DF4F0FB66D
:1005D000F894DEBF0FBECDBFDF91CF911F9108957C
:1005E000133081F060911601709117011430E9F613
:1005F000CE0101960E944516D8CF60911A017091E4
:100600001B01F6CF6091180170911901F1CFDC0147
:10061000FB019C918081981311C011969C911197B8
:10062000818198130BC012969C9112978281981326
:1006300005C081E013962C919381291380E00895E1
:100640000F931F93CF9322E040E1609104018BEE62
:1006500092E00E94E40588ED92E00E94CF05E8ED6B
:10066000F2E008E711E011830083C1E0C28B85EC62
:1006700092E00E94CF05E5ECF2E011830083C28B8B
:1006800082EB92E00E94CF05E2EBF2E0118300835F
:10069000C28B8FE992E00E94CF05EFE9F2E011836F
:1006A0000083C28B68ED72E083E592E00E94A100B6
:1006B00065EC72E086E692E00E94A10062EB72E0D7
:1006C00089E792E00E94A1006FE972E08CE892E075
:1006D0000E94A10080E592E00E94960A40E16EE04F
:1006E00080E492E00E948C0C40E16FE080E392E0B5
:1006F000CF911F910F910C948C0CFF920F931F932D
:10070000CF93DF93C3E5D2E010E000E0CE010E947A
:100710006205888582FF20C0CE010E94CB059A89A0
:1007200089131AC060910803F801E458FE4FF08065
:10073000E62FF0E0E75FFC4FF08241E08BEE92E0C5
:100740000E9462066F2D8BEE92E00E949A068091C5
:1007500008038F5F809308038BEE92E00E9454069B
:1007600040E062E08BEE92E00E94620665E071E09C
:100770008BEE92E00E94241441E060E08BEE92E068
:100780000E94620669E073E08BEE92E00E942414FE
:100790008BEE92E00E940E066EE170E080E090E049
:1007A0000E94D4110F5F1F4F63960430110509F0AA
:1007B000ADCF80910803883009F040C062E271E05B
:1007C00089E093E00E94B301109208038FE58093C3
:1007D000090380930A0380930B0380930C03809397
:1007E0000D0380930E0380930F03809310038BEE11
:1007F00092E00E94540640E062E08BEE92E00E949C
:10080000620665E071E08BEE92E00E94241441E004
:1008100060E08BEE92E00E94620669E073E08BEE8E
:1008200092E00E9424146EE170E080E090E0DF919D
:10083000CF911F910F91FF900C94D411DF91CF9124
:100840001F910F91FF9008950F931F930E94A31182
:100850000091FB021091FC022091FD023091FE02FA
:10086000601B710B820B930B603177428105910500
:1008700078F08091FA0281110BC01092040310925B
:100880000503109206031092070381E08093FA0299
:1008900080E492E00E94E21090E090930203809343
:1008A000010380E492E00E94FC0B282F30E030939B
:1008B00000032093FF022091010330910203232BB8
:1008C00009F452C0882309F44FC0809143028093F9
:1008D0000403809144028093050380914502809334
:1008E000060380914602809307031092FA0280E487
:1008F00092E00E94121180E492E00E9455110E9441
:10090000A3116093FB027093FC028093FD0290930D
:10091000FE0264E073E08EE191E00E9407038093A1
:10092000030381110DC081E00E94950160ED77E025
:1009300080E090E00E94D4111F910F910C948D01E2
:100940008130A9F482E00E94950168EB7BE080E0B1
:1009500090E00E94D4110E948D01809101018330AA
:1009600019F484E0809301011F910F910895823062
:10097000D9F783E00E94950164EF71E080E090E098
:10098000D9CF8AE00E943013892B79F484E00E9449
:1009900030130197B1F460E084E00E94021360ED2F
:1009A00077E080E090E00E94D41181E10E94301352
:1009B0008093F90281110AC080910101813079F49C
:1009C0000895809101010E94A402EFCF813039F493
:1009D00080910101813019F482E08093010182E06D
:1009E0000E9430138093F80290910101811103C09D
:1009F000923041F40895813029F4923019F483E063
:100A00008093010180910101833011F40E9424043C
:100A100080910101843031F48BEE92E00E940E0649
:100A20000E947D03909101018091000198131EC0E6
:100A30008BEE92E00E9454068BEE92E00E940E062E
:100A400040E060E08BEE92E00E9462066DE571E0AE
:100A50008BEE92E00E94241461E084E00E94021375
:100A60006EE170E080E090E00C94D4110895FC01F8
:100A700082E791E09183808312821382148215822F
:100A80008AE090E09783868310860895FC0177833F
:100A900066830895CF93DF93EC011886E881F9818E
:100AA0000190F081E02D0995882319F088858360F5
:100AB00088870E94A3116A837B838C839D83DF9147
:100AC000CF910895CF92DF92EF92FF920F931F93F1
:100AD000CF93DF93EC0188858B7F8887E881F9814C
:100AE0000190F081E02DCE010995182F888586951B
:100AF00081701817B9F00E94A3116A837B838C83DD
:100B00009D83888592E089278887888582FB88274E
:100B100080F9DF91CF911F910F91FF90EF90DF90BF
:100B2000CF9008950E94A311CA80DB80EC80FD80E5
:100B3000AB01BC014C195D096E097F098E819F8153
:100B4000B0E0A0E0481759076A077B07F0F28885F4
:100B500081701817D1F20E94A3116A837B838C8362
:100B60009D83888591E08927846088870E94A311EE
:100B700009851A852B853C85601B710B820B930BB5
:100B80006D877E878F87988B0E94A31169877A87EC
:100B90008B879C87BACFFC01808581700895CF93A5
:100BA000DF93EC010E94370581EF91E09983888300
:100BB000198ADF91CF910895FC01618B0C944A054D
:100BC00090E080E008950895FC011382128289EF7D
:100BD00091E09183808364834187228713860895FF
:100BE0000F931F93CF938C01C62FFC01648182E188
:100BF00093E00E94D407F80163856C2B82E193E0B7
:100C00000E94660782E193E0CF911F910F910C94AF
:100C1000F107FC01138660E00C94F00528E0FC016C
:100C2000238760E00C94F0050F931F93CF938C0102
:100C3000C62F64600E94F00581E090E00E940D12D2
:100C40006C2F6B7FC8010E94F00582E390E0CF918A
:100C50001F910F910C940D121F93CF93DF93EC0112
:100C6000162F0E94F005612FCE01DF91CF911F91C9
:100C70000C9414060F931F93CF93DF938C01D62F00
:100C8000C42F607F642B0E942C0680E1D89FB001A6
:100C900011246C2BC801DF91CF911F910F910C94FF
:100CA0002C0640E00C943A0661E00E94510680ED6B
:100CB00097E00C940D1262E00E94510680ED97E0DF
:100CC0000C940D12CF93DF93CDB7DEB728970FB6F4
:100CD000F894DEBF0FBECDBF28E0EBE2F1E0DE010D
:100CE000119601900D922A95E1F7FC0120852417B9
:100CF00010F44FEF420F50E0440F551F21E030E059
:100D00002C0F3D1F420F531FFA012081620F6068B4
:100D100028960FB6F894DEBF0FBECDBFDF91CF91FE
:100D20000C945106FC016681262F246026836C609A
:100D30000C94510641E00E943A0681E090E008954B
:100D4000CF93DF93EC01423018F08D8188608D8362
:100D50004887222329F0413019F48D8184608D83E6
:100D600062E370E080E090E00E94D4116B85CE01D8
:100D70000E94F00568EE73E080E090E00E94D411DC
:100D800060E3CE010E942C0684E991E10E940D12DD
:100D900060E3CE010E942C0684E991E10E940D12CD
:100DA00060E3CE010E942C0686E990E00E940D12BD
:100DB00060E2CE010E942C066D816062CE010E942D
:100DC000510684E08E83CE010E949206CE010E94DD
:100DD000540682E08F8366E0CE010E945106CE0168
:100DE000DF91CF910C945B06CF93DF93EC0182E10E
:100DF00093E00E94C2071D8220E04A856985CE01EA
:100E0000DF91CF910C94A0060C94F40680914603D8
:100E100090914703891B990B089590914703809106
:100E200046032FEF3FEF981748F4E92FF0E0E85B17
:100E3000FC4F208130E09F5F90934703C9010895E4
:100E4000E091470380914603E81730F4F0E0E85B57
:100E5000FC4F808190E008958FEF9FEF08950895F3
:100E6000CF93DF93EC01E0911E03F0911F033097C5
:100E7000F1F090914703809146039817C0F090E0FD
:100E8000292F30E02617370754F4DE01A20FB31FD5
:100E90004C91285B3C4FD9014C939F5FF1CF10924E
:100EA000470360934603CB01DF91CF910994DF9113
:100EB000CF910895E0912003F0912103309729F01C
:100EC000109224031092230309940895CF93DF9383
:100ED0001F92CDB7DEB76983209122032223F9F058
:100EE00020912303203258F021E030E0FC013383CD
:100EF000228390E080E00F90DF91CF910895809160
:100F00002403E82FF0E0EB5DFC4F998190838F5F25
:100F1000809324038093230381E090E0ECCF61E091
:100F2000CE0101960E947A08F7CFCF92DF92EF921E
:100F3000FF920F931F93CF93DF937C01CB018A0124
:100F400020912203222389F0EB016B01C40ED51EF0
:100F5000CC15DD0569F06991D701ED91FC91019007
:100F6000F081E02DC7010995F3CF642F0E947A0824
:100F7000C801DF91CF911F910F91FF90EF90DF900B
:100F8000CF900895109247031092460310922403C5
:100F9000109223030E9405088AE597E00E94A608A4
:100FA00080E397E00C94A10881E080932203609392
:100FB0004503109224031092230308950F93062FE4
:100FC00021E04091230365E273E0809145030E9494
:100FD00023081092240310922303109222030F91EE
:100FE000089561E00C94DE07E2E1F3E013821282DF
:100FF00088EE93E0A0E0B0E084839583A683B78376
:1010000085E092E09183808308951092D50381E07A
:101010008093D3031092D20361E082E10E94021315
:1010200061E083E10E940213E9EBF0E080818E7FB2
:10103000808380818D7F808380E28093B80085E407
:101040008093BC0008950F93413208F04BC09091FB
:10105000D5039111FCCF92E09093D5030093D30375
:101060009FEF909368031092AD034093AC03362F2B
:10107000AEEAB3E0FB019E2F931B941770F1109220
:10108000D4039091D403880F892B8093D40380914B
:10109000D203813029F51092D2038091D40380933A
:1010A000BB008091BC0083FDF8CF85EC8093BC0031
:1010B000222321F08091D5038230D1F380916803FF
:1010C0008F3F91F080916803803281F080916803B6
:1010D000803371F084E00F91089591919D93CBCF6F
:1010E00085EEE4CF81E0F7CF80E0F5CF82E0F3CF6B
:1010F00083E0F1CF20918A03260F3327331F21325B
:101100003105ECF42091D503FC0190E080E024301F
:1011100069F082E00895A0918A032191AC014457BF
:101120005C4FA40FB52FB11D2C930196861798F331
:1011300080918A03680F60938A0380E0089581E0BC
:1011400008959093CF038093CE0308959093D10395
:101150008093D003089585ED8093BC008091BC00FE
:1011600084FDFCCF1092D503089585EC8093BC00DC
:101170001092D50308951F920F920FB60F9211246B
:101180002F933F934F935F936F937F938F939F938F
:10119000AF93BF93EF93FF938091B900887F803620
:1011A00009F44CC008F03FC0883209F4A8C018F513
:1011B000803109F49CC0B8F4882309F4F9C0883060
:1011C00009F495C0FF91EF91BF91AF919F918F91DD
:1011D0007F916F915F914F913F912F910F900FBE33
:1011E0000F901F901895883109F489C0803251F70B
:1011F0008093680315C0803409F49EC048F480339E
:10120000B9F38833F9F6809368030E94B508DACF02
:10121000803509F485C0883509F496C0883491F684
:101220000E94AB08CFCF883909F48CC038F58837D5
:1012300029F050F4883611F0803721F683E080934E
:10124000D5031092690357C0883809F47BC08039F0
:1012500019F0803809F0B6CF80916903803208F028
:1012600071C0E091690381E08E0F809369038091E2
:10127000BB00F0E0E659FC4F80833DC0803B39F075
:10128000E0F4803A09F479C0883A09F09BCF84E011
:101290008093D50310928B0310928A03E091D003C0
:1012A000F091D103099580918A0381110FC081E0EB
:1012B00080938A0310928C0309C0803C09F476C0A5
:1012C000883C09F473C0883B09F07CCFE0918B0324
:1012D00081E08E0F80938B03F0E0E457FC4F808118
:1012E0008093BB0090918B0380918A0329C08091E9
:1012F000D4038093BB0085EC8093BC0063CF9091B6
:10130000AD038091AC03981758F5E091AD0381E0EF
:101310008E0F8093AD03F0E0E255FC4F8081E9CF62
:10132000E091AD0381E08E0F8093AD038091BB000F
:10133000F0E0E255FC4F80839091AD038091AC03C7
:101340009817C8F285E8D8CFE091AD0381E08E0F01
:101350008093AD038091BB00F0E0E255FC4F8083A9
:101360008091D30381115CCF81E08093D20384EA22
:101370008093BC001092D50325CF0E94B5088091C0
:101380006903803230F4E0916903F0E0E659FC4FE4
:1013900010826091690370E0E091CE03F091CF0379
:1013A0008AE693E00995109269030CCF85ECE0CFB3
:1013B0001092680335CF1F920F920FB60F9211242F
:1013C0002F933F934F935F936F937F938F939F934D
:1013D000AF93BF93EF93FF938091D70387FF27C00D
:1013E00010928500109284008091D7038F5F8093C4
:1013F000D7038091D703082E000C990B2091D603B8
:101400002817190629F024F08091D7038C30DCF1DD
:101410008091840090918500049680329E4408F467
:101420007BC08091840090918500049677C0809164
:10143000D703082E000C990B2091D6032817190604
:1014400099F294F2E091D7038E2FEE0F990BFC01E5
:10145000EE0FFF1FE80FF91FE852FC4F808186FF57
:10146000C3CFE091D7038E2FEE0F990BFC01EE0F47
:10147000FF1FE80FF91FE852FC4F808160E08F7377
:101480000E940213B1CF2091840030918500E09139
:10149000D7038E2FEE0F990BFC01EE0FFF1FE80F05
:1014A000F91FE852FC4F81819281820F931F909324
:1014B000890080938800E091D7038E2FEE0F990B5F
:1014C000FC01EE0FFF1FE80FF91FE852FC4F80816F
:1014D00086FF11C0E091D7038E2FEE0F990BFC0110
:1014E000EE0FFF1FE80FF91FE852FC4F808161E00B
:1014F0008F730E940213FF91EF91BF91AF919F9163
:101500008F917F916F915F914F913F912F910F90AC
:101510000FBE0F901F90189580E29EE49093890073
:10152000809388008FEF8093D703E5CFFC019091E3
:10153000D6039C3098F481E0890F8093D603908382
:10154000892F90E0FC01EE0FFF1FE80FF91FE85212
:10155000FC4F8CED95E09283818308958FEF80831B
:101560000895DF92EF92FF920F931F93CF93DF9333
:10157000EC01D62E7A01890188818C3008F067C091
:1015800061E08D2D0E94C6128881282F30E0F9017C
:10159000EE0FFF1FE20FF31FE852FC4F9D2D9F73CC
:1015A0006081607C692B608320E232E02E193F0964
:1015B00037FF02C02D5F3F4F35952795359527950D
:1015C000298320E639E0201B310B37FF02C02D5F55
:1015D0003F4F35952795359527952A832CE0622F27
:1015E0000E94CA15829FB001112430E020E0AB01B7
:1015F000420F531FFA01EE0FFF1FE40FF51FE852D1
:10160000FC4F908196FD16C02F5F3F4F2C30310567
:1016100071F781110FC01092800082E080938100E9
:101620001092850010928400B19A80916F008260C0
:1016300080936F00E8818E2F90E0FC01EE0FFF1F7A
:10164000E80FF91FE852FC4F808180648083888115
:10165000DF91CF911F910F91FF90EF90DF90089550
:1016600020E639E040E252E00C94B10ADC01EC9152
:10167000EC3080F511968C91119728E830E0281B0A
:10168000310987FD3395220F331F220F331F621755
:10169000730784F012968C9128E532E0281B3109FB
:1016A00087FD3395220F331F220F331F62177307F5
:1016B0000CF49B014FB7F8948E2F90E02250310923
:1016C000FC01EE0FFF1FE80FF91FE852FC4F3283B9
:1016D00021834FBF0895AF92BF92CF92DF92EF92D6
:1016E000FF920F931F93CF93DF93EC01603282E060
:1016F00078070CF03EC0653B710514F064EB70E0B8
:10170000898148E8A42EB12CA81AB10887FDB394AA
:10171000AA0CBB1CAA0CBB1C0B2C000CCC08DD08B3
:1017200077FF02C070E060E0072E000C880B990B79
:101730002A8108E512E0021B110927FD1395000F0D
:10174000111F000F111F012E000C220B330B3F93B2
:101750002F931F930F9314EBE12EF12C00E010E078
:1017600020E030E0A9010E9493140F900F900F9099
:101770000F90CE01DF91CF911F910F91FF90EF90CD
:10178000DF90CF90BF90AF900C94360BCF93CFB734
:10179000F8948091FF03811127C0E0EAF0E0849182
:1017A000E9E8F0E09491E82FF0E0EE0FFF1FEF532F
:1017B000FF4FA591B491EC91E92321F461E08AE017
:1017C0000E94021361E08AE00E94C6128CB580611B
:1017D0008CBD8CB580648CBD61E08DE00E94C6122A
:1017E00061E08BE00E94C6128091FF038F5F8093BF
:1017F000FF03CFBFCF910895BC016E5F7F4FDC0127
:10180000ED91FC910190F081E02D40E0099591E08F
:10181000811190E0892F08952091FE03222381F009
:101820003FB7F8942091FE03213069F42DB3209343
:10183000FC034DB32091FD03209524232DBB3FBF16
:101840008CBD9DBD08953093FC03FACF8EBD000082
:101850000DB407FEFDCF8EB508958091FE03882359
:1018600061F09FB7F8942091FE038091FC03213032
:1018700019F48DBB9FBF08958FBF0895CF92DF925B
:10188000EF92FF920F931F93CF93DF937C01C42EAF
:10189000E901D62E6894D7F880E591E00E940C0CFF
:1018A00060E0F70186850E940213CA948D2D0E9484
:1018B000260C0023A1F08FEF90E09C0102C0220FC4
:1018C000331F0A95E2F789018D2D0E94260C902F77
:1018D0009095288192238023892B888301E0C00F73
:1018E000D11D0C1530F48D2D0E94260C89930F5FAD
:1018F000F8CF80E00E94260C888361E0F70186859E
:101900000E940213DF91CF911F910F91FF90EF90F2
:10191000DF90CF900C942D0CFC0187E192E0918335
:1019200080836687478708950F931F93CF93DF9334
:10193000EC01062F142F80E591E00E940C0C60E072
:101940008E850E940213802F0E94260C812F0E94F8
:10195000260C61E08E850E940213DF91CF911F91CA
:101960000F910C942D0CDF92EF92FF920F931F9327
:10197000CF93DF937C01C62F042FD22E132F80E547
:1019800091E00E940C0C60E0F70186850E94021332
:101990008C2F0E94260CCD2DD12F0C0F1D2F111D29
:1019A000C017D10721F089910E94260CF9CF61E080
:1019B000F70186850E940213DF91CF911F910F914D
:1019C000FF90EF90DF900C942D0C1F93CF93DF933B
:1019D000EC01162F80E591E00E940C0C60E08E85F2
:1019E0000E940213812F80680E94260C80E00E94D2
:1019F000260C182F61E08E850E9402130E942D0C88
:101A0000812FDF91CF911F9108950F9341110E9473
:101A10003E0C0F9108950F931F93CF93DF938C018A
:101A2000D62FC42F0E94E50C482F4C2B6D2FC801D8
:101A3000DF91CF911F910F910C94940C0F931F93F2
:101A4000CF93DF938C01D62FC42F0E94E50CC09555
:101A50004C2F48236D2FC801DF91CF911F910F911B
:101A60000C94940CCF92DF92EF92FF920F931F93FE
:101A7000CF93DF93EC016B01142F790140E062E01A
:101A80000E94940C44E06AE0CE010E94940C40E86D
:101A900064E1CE010E94940C9601412F62E1CE01D7
:101AA0000E94B30C43E062E0CE010E94940C08E86F
:101AB00013E16AE0CE010E94E50C82FF1BC040E00A
:101AC00062E0CE010E94940C64E4CE010E94E50C19
:101AD000F701808362E4CE010E94E50CF701818367
:101AE00080E0DF91CF911F910F91FF90EF90DF90F9
:101AF000CF90089501501109E1F683E0F2CF0F93E2
:101B00001F93CF938C014FE062E00E94940CC3E0DE
:101B100062E370E080E090E00E94D41162E0C801CE
:101B20000E94E50C84FF02C0C15091F7CF911F9134
:101B30000F910895CF93DF93EC0168E20E94E50CCA
:101B4000982F9370933041F0482F436068E2CE01A4
:101B5000DF91CF910C94940CDF91CF910895CF93A6
:101B6000DF93EC0161E08E850E94C61261E08E85F4
:101B70000E9402138F858F3F09F451C060E00E94DC
:101B8000C6128F850E943013892B09F048C061E08E
:101B90008F850E94C61260E08F850E94021382E04A
:101BA00090E00E940D1261E08F850E94021362E3B3
:101BB00070E080E090E00E94D41140E064E2CE0149
:101BC0000E94940C40E066E2CE010E94940C46E232
:101BD00068E4CE010E94940C40E864E5CE010E94C6
:101BE000940C49EA66E5CE010E94940C43E068E556
:101BF000CE010E94940C48EE6AE5CE010E94940C3E
:101C000040E46AE2CE010E94940C4DE362E2CE0110
:101C10000E94940CCE01DF91CF910C949A0DCE01CD
:101C20000E947F0DCACF3F924F925F926F927F9238
:101C30008F929F92AF92BF92CF92DF92EF92FF92DC
:101C40000F931F93CF93DF9300D0CDB7DEB73C0146
:101C5000162F942E290180E0A114B10411F0F50192
:101C60008081382C329490EF3922380E40E062E0C7
:101C7000C3010E94940C4FE768E0C3010E94940CDA
:101C800040E864E1C3010E94940C9201402F62E19C
:101C9000C3010E94B30C432D6AE1C3010E94940C5E
:101CA000412F62E0C3010E94940C1C3029F440E8EB
:101CB0006AE1C3010E940B0D00ED17E068E0C3016B
:101CC0000E94E50C982F992109F07BC080FD03C08C
:101CD0000150110999F783E038C0E114F10409F4C7
:101CE00048C0C114D10409F444C064E1C3010E9496
:101CF000E50CF6019081981708F45FC08083082DE9
:101D00009701482F62E1C3010E94050D68E1C301FC
:101D10000E94E50C8770A114B10411F0F5018083D5
:101D200013FD4DC0E114F10409F445C0C114D10400
:101D300009F441C09E899923F1F1F60140814130B7
:101D4000D1F4843009F047C08FEF0F900F90DF91EE
:101D5000CF911F910F91FF90EF90DF90CF90BF90A8
:101D6000AF909F908F907F906F905F904F903F903B
:101D7000089580E0D5CF423070F181112CC04250DF
:101D80009E012F5F3F4FB701C3010E94320D8111A9
:101D9000DCCFF6018081E80EF11CF70132979081CB
:101DA0008981981318C0F1E0EF1AF108F7019081CA
:101DB0008A81981310C080E0C8CF84E0C6CF82E04B
:101DC000C4CF6CE0C3010E94E50C182F837109F4A5
:101DD00084CF81E0BACF87E0B8CF8F92AF92BF9225
:101DE000CF92DF92EF92FF920F931F93AF928C2CC2
:101DF000570168017901042F9B0140E36CE00E94C8
:101E0000130E0F901F910F91FF90EF90DF90CF90E6
:101E1000BF90AF908F9008952F923F924F925F9214
:101E20006F927F928F929F92AF92BF92CF92DF92EA
:101E3000EF92FF920F931F93CF93DF93CDB7DEB74F
:101E40002D970FB6F894DEBF0FBECDBF16E041351B
:101E500008F045C1342E4B013C0140E86CE10E9482
:101E60001E0D83E98983332029F081E0F4019081FC
:101E7000953008F480E022242394B12C9B2D990FF7
:101E8000990F990FD32CD91AD7FCD12C32E0882383
:101E900019F098E89B8333E021E09D2D977009F4B9
:101EA00020E09D2D959595959595290FC9F094E085
:101EB000811193E0291708F4922FEB2DF0E0319671
:101EC000E80DF91D232F4191A1E0B0E0AC0FBD1F3B
:101ED000A20FB11D4C932F5F422F431B491798F35C
:101EE000882311F0F8E0DF0E8FE18D150CF082C031
:101EF00090E79A838B819C8189279D8189279E8188
:101F000089278F839E01285F3F4F47E0BE016F5FA7
:101F10007F4FC3010E94320D182F8111E0C01B8634
:101F2000E3E0EA87DC86CE0107962C0199E09D87E5
:101F3000CB844C2D4295407F4C0D6AE1C3010E9439
:101F4000940CA12CCE010B967C018E01065F1F4FD5
:101F500092014D85BE016F5F7F4FC3010E94ED0E60
:101F6000182F823009F065C06CE1C3010E94E50CB6
:101F700085FDB5C08F7109F480E2282F30E04D2D2A
:101F8000DD0C550B421753070CF09DC0D82EE82FDF
:101F9000E595E595E595EF5F982F977081E009F459
:101FA00080E0E80F81E090E08C0F9D1F8E0F911D67
:101FB000FC01215031092770332781E090E002C0F5
:101FC000880F991F2A95E2F79C018081822B8083DC
:101FD0008BCF85E98983332031F081E0F401908152
:101FE000983008F04BCF80E049CF87E9898326E01D
:101FF000B22EF9CF9D2D97709B878D2D8595859558
:1020000085958E5F282F2295207F290F2A8321E036
:10201000911101C020E0280F2D8744244394512CB6
:102020004C0E5D1E480E511CE9E0E81BEA87DC8679
:102030007FCF811154C080E2D82E9C8590320CF461
:1020400057CF8B81883809F040C083E093E0EB2DB7
:10205000F0E03196E80DF91D980FA1E0B0E0AC0F6B
:10206000BD1FA80FB11D2C9121938F5F8913F5CF50
:10207000BA84E3E0BE124DC08B8581114AC09E0137
:102080002D5F3F4F41E0B201C3010E94320D182F76
:10209000811125C09B81F201818198133CC09C81F4
:1020A0008281981338C0808182FF12C02394F2E0AD
:1020B0002F1609F48ECF83E0281609F496CF91E00D
:1020C000291609F4CECE15E00AC082E094E0BFCF15
:1020D000F4018387822D880F820D8F5F8083812F8B
:1020E0002D960FB6F894DEBF0FBECDBFDF91CF9116
:1020F0001F910F91FF90EF90DF90CF90BF90AF9026
:102100009F908F907F906F905F904F903F902F9017
:10211000089511E0E4CF17E0E2CF4F925F926F9203
:102120007F928F929F92AF92CF92EF92FF920F93F6
:102130001F93CF93DF9300D0CDB7DEB76A834115ED
:102140005105B9F1F9016081623098F149012A0124
:102150003C0140E86CE10E941E0D87E08983A12CC0
:10216000C12CCE0101967C018401920141E0BE01A7
:102170006E5F7F4FC3010E94ED0E811109C0F40113
:1021800080818230C1F481E09981911101C080E0A9
:102190000F900F90DF91CF911F910F91FF90EF90D3
:1021A000CF90AF909F908F907F906F905F904F9067
:1021B000089584E0EDCF81E0EBCF9A01AB0166E2B8
:1021C0000C948D100F931F93CF93DF9300D01F9229
:1021D000CDB7DEB78C0182E08B8340E064E2C801BA
:1021E0000E94940C40E066E2C8010E94940C46E212
:1021F00068E4C8010E94940CAE014D5F5F4FBE01C0
:102200006F5F7F4FC8010E94DD10982F9D7F81E096
:1022100009F080E00F900F900F90DF91CF911F9108
:102220000F9108958F929F92AF92CF92EF92FF926B
:102230000F931F93CF93DF9300D000D0CDB7DEB7BD
:102240004C0180E589831A829E012D5F3F4F42E059
:10225000BE016F5F7F4FC4010E94320D811116C015
:10226000A12CC12CF12CE12C10E000E030E020E0AA
:1022700044E0BE016F5F7F4FC4010E94ED0E8330CA
:1022800021F0811103C081E001C080E00F900F9028
:102290000F900F90DF91CF911F910F91FF90EF90D2
:1022A000CF90AF909F908F90089548E060E10C949C
:1022B0001E0D1F920F920FB60F9211242F933F9372
:1022C0008F939F93AF93BF938091050490910604E1
:1022D000A0910704B09108043091040426E0230F74
:1022E0002D3768F129E8230F0396A11DB11D209316
:1022F00004048093050490930604A0930704B0930C
:1023000008048091000490910104A0910204B0910E
:1023100003040196A11DB11D809300049093010454
:10232000A0930204B0930304BF91AF919F918F914A
:102330003F912F910F900FBE0F901F90189502960E
:10234000A11DB11DD4CF2FB7F894609105047091F1
:10235000060480910704909108042FBF08953FB7A9
:10236000F8948091000490910104A0910204B0912E
:10237000030426B5A89B05C02F3F19F00196A11DA7
:10238000B11D3FBFBA2FA92F982F8827BC01CD01BF
:10239000620F711D811D911D43E0660F771F881F1D
:1023A000991F4A95D1F708958F929F92AF92BF924D
:1023B000CF92DF92EF92FF926B017C010E94AF11EE
:1023C0004B015C01C114D104E104F104E9F00E9465
:1023D000E6140E94AF11681979098A099B09683EC1
:1023E00073408105910570F321E0C21AD108E1081C
:1023F000F10888EE880E83E0981EA11CB11CC11460
:10240000D104E104F10429F7FF90EF90DF90CF9021
:10241000BF90AF909F908F90089500000000833090
:10242000910528F0880F991F05970197F1F70895F6
:10243000789484B5836084BD85B5836085BDEEE600
:10244000F0E0808181608083E1E8F0E082E08083D9
:10245000808181608083E0E8F0E08081816080831A
:10246000E1EBF0E0808184608083E0EBF0E080814C
:102470008160808386E880937A001092C10008957D
:102480001F93CF93DF93182FEB0161E00E94C612D8
:10249000209739F460E0812FDF91CF911F910C9448
:1024A0000213CF3FD10511F461E0F5CFE12FF0E049
:1024B000E859FF4FE491E43031F140F4E230B1F0FB
:1024C000E330E1F0C038D1057CF7E4CFE83029F102
:1024D000E93059F1E530B1F7809180008062809356
:1024E0008000D0938B00C0938A0004C084B58068BC
:1024F00084BDC7BDDF91CF911F91089584B58062DF
:1025000084BDC8BDF7CF8091800080688093800033
:10251000D0938900C0938800EDCF8091B00080688F
:102520008093B000C093B300E5CF8091B00080628B
:102530008093B000C093B400DDCF843081F028F4E4
:102540008230E9F08330F9F00895883071F08930F5
:1025500091F08530B9F4809180008F7D03C0809127
:1025600080008F778093800008958091B0008F77EE
:102570008093B00008958091B0008F7DF9CF84B52D
:102580008F7784BD089584B58F7DFBCFCF93DF9384
:1025900090E0FC01E158FF4F24918A569F4FFC01C7
:1025A00084918823C9F090E0880F991FFC01EF53B4
:1025B000FF4FA591B491FC01E954FF4FC591D4910F
:1025C00061110DC09FB7F8948C91209582238C9354
:1025D0008881282328839FBFDF91CF91089562309F
:1025E00051F49FB7F8943C91822F809583238C936C
:1025F000E8812E2BEFCF8FB7F894EC912E2B2C93F4
:102600008FBFEACF1F93CF93DF93282F30E0F901DC
:10261000E859FF4F8491F901E158FF4FD491F90136
:10262000EA56FF4FC491CC23A9F0162F81110E94C6
:102630009D12EC2FF0E0EE0FFF1FE954FF4FA59124
:10264000B4918FB7F894EC91111108C0D095DE23A6
:10265000DC938FBFDF91CF911F910895DE2BF8CFD0
:10266000CF93DF93282F30E0F901E859FF4F849191
:10267000F901E158FF4FD491F901EA56FF4FC49197
:10268000CC23A1F081110E949D12EC2FF0E0EE0FFF
:10269000FF1FE355FF4FA591B491EC91ED2381E02D
:1026A00090E009F480E0DF91CF91089580E090E020
:1026B000FACF1F920F920FB60F9211242F938F9380
:1026C0009F93EF93FF93E0911904F0911A04808196
:1026D000E0911F04F091200482FD1BC09081809145
:1026E00022048F5F8F7320912304821741F0E091C1
:1026F0002204F0E0E75FFB4F958F80932204FF9167
:10270000EF919F918F912F910F900FBE0F901F907F
:1027100018958081F4CF1F920F920FB60F9211245B
:102720002F933F934F935F936F937F938F939F93D9
:10273000AF93BF93EF93FF9389E094E00E9432152B
:10274000FF91EF91BF91AF919F918F917F916F9189
:102750005F914F913F912F910F900FBE0F901F905F
:10276000189589E094E00E94E71421E0892B09F490
:1027700020E0822F0895E9E0F4E01382128288EECF
:1027800093E0A0E0B0E084839583A683B78381E2E1
:1027900092E09183808385EC90E09587848784EC38
:1027A00090E09787868780EC90E0918B808B81EC1E
:1027B00090E0938B828B82EC90E0958B848B86ECFF
:1027C00090E0978B868B118E128E138E148E089547
:1027D000AF92BF92CF92DF92EF92FF920F931F932F
:1027E000CF93DF936C017B018B01040F151FEB016D
:1027F0005E01AE18BF08C017D10759F06991D60124
:10280000ED91FC910190F081E02DC6010995892B95
:1028100079F7C501DF91CF911F910F91FF90EF9054
:10282000DF90CF90BF90AF900895FB010190002002
:10283000E9F73197AF01461B570BDC01ED91FC9195
:102840000280F381E02D09946115710511F00C945B
:10285000151490E080E00895DC01ED91FC91019069
:10286000F081E02D09948F929F92AF92BF92EF92E8
:10287000FF920F931F93CF93DF93CDB7DEB7A1974E
:102880000FB6F894DEBF0FBECDBF7C01FA01CB01BD
:1028900019A2223008F42AE08E010F5D1F4F822E0C
:1028A000912CB12CA12CBF01A50194010E94D61539
:1028B000F901CA016A300CF5605DD8016E938D0193
:1028C000232B242B252B79F790E080E0109721F023
:1028D000BD01C7010E941514A1960FB6F894DEBF82
:1028E0000FBECDBFDF91CF911F910F91FF90EF9061
:1028F000BF90AF909F908F900895695CDECF2115B7
:10290000310541F4DC01ED91FC910190F081E02D65
:10291000642F09940C9433149A01462F50E070E010
:1029200060E00C947F144F925F926F927F92AF920F
:10293000BF92CF92DF92EF92FF920F931F93CF93AC
:10294000DF93CDB7DEB729013A019B01AC01241911
:1029500035094609570989899A89AB89BC89BC011F
:10296000CD016A197B098C099D090E94BA15A8013D
:10297000970124193509460957090E94F815CA011B
:10298000B9016A0D7B1D8C1D9D1DDF91CF911F919B
:102990000F91FF90EF90DF90CF90BF90AF907F901E
:1029A0006F905F904F9008950E94371608950E948F
:1029B00018120E94D6140E94DB00C4E2D5E10E94E6
:1029C000C1042097E1F30E942415F9CF0895FC017A
:1029D000918D228D892F90E0805C9F4F821B910901
:1029E0008F7399270895FC01918D828D981731F08E
:1029F000828DE80FF11D858D90E008958FEF9FEF98
:102A00000895FC01918D828D981761F0A28DAE0F13
:102A1000BF2FB11D5D968C91928D9F5F9F73928F9A
:102A200090E008958FEF9FEF0895FC01538D448D42
:102A3000252F30E0842F90E0821B930B541710F069
:102A4000CF9608950197089581EB93E1892B49F082
:102A500080E090E0892B29F00E94B11381110C9441
:102A600000000895FC01A48DA80FB92FB11DA35A31
:102A7000BF4F2C91848D90E001968F739927848F9E
:102A8000A689B7892C93A089B1898C9180648C9395
:102A9000938D848D981306C00288F389E02D808180
:102AA0008F7D80830895CF93DF93EC01888D8823F9
:102AB000B9F0AA89BB89E889F9898C9185FD03C0A1
:102AC000808186FD0DC00FB607FCF7CF8C9185FF86
:102AD000F2CF808185FFEDCFCE010E943215E9CF84
:102AE000DF91CF910895EF92FF920F931F93CF93B1
:102AF000DF93EC0181E0888F9B8D8C8D981316C03D
:102B0000E889F989808185FF11C0EE89FF8960839A
:102B1000E889F98980818064808381E090E0DF9199
:102B2000CF911F910F91FF90EF900895F62E0B8D8E
:102B300010E00F5F1F4F0F731127E02E8C8D8E1149
:102B40000CC00FB607FCFACFE889F989808185FFB0
:102B5000F5CFCE010E943215F1CFEB8DEC0FFD2F9A
:102B6000F11DE35AFF4FF0820B8FEA89FB898081C8
:102B70008062D2CFDB018F939F930E941D16BF917D
:102B8000AF91A29F800D911DA39F900DB29F900DBC
:102B900011240895991B79E004C0991F961708F035
:102BA000961B881F7A95C9F780950895A1E21A2E81
:102BB000AA1BBB1BFD010DC0AA1FBB1FEE1FFF1FE1
:102BC000A217B307E407F50720F0A21BB30BE40B31
:102BD000F50B661F771F881F991F1A9469F7609578
:102BE0007095809590959B01AC01BD01CF01089532
:102BF000052E97FB1EF400940E940F1657FD07D078
:102C00000E94D61507FC03D04EF40C940F16509575
:102C10004095309521953F4F4F4F5F4F08959095C8
:102C20008095709561957F4F8F4F9F4F0895EE0F60
:102C3000FF1F0590F491E02D09940E942816A59F8E
:102C4000900DB49F900DA49F800D911D11240895A7
:102C5000A29FB001B39FC001A39F700D811D1124DD
:102C6000911DB29F700D811D1124911D089581E069
:102C700090E0F8940C944C16FB01DC018D910190CE
:102C800080190110D9F3990B0895FB01DC01019023
:0C2C90000D920020E1F70895F894FFCFAA
:102C9C000501781E2741636365737320436F646578
:102CAC003F000000000085019F01B901D3018A3764
:102CBC00F280415443474743544100000040001404
:102CCC0000540041636365737300417574686F72DF
:102CDC00697A6564210044656E6965642100486504
:102CEC006C70202D2050757A7A6C652000436F6EC5
:102CFC0067726174756C6174696F6E73210000008A
:102D0C000000D41400000000970093004143544786
:102D1C005F1407150848656C70206D6573736167E7
:102D2C006520666F722070757A7A6C652034004865
:102D3C00656C70206D65737361676520666F7220BA
:102D4C0070757A7A6C6520330048656C70206D65FF
:102D5C00737361676520666F722070757A7A6C6523
:102D6C0020320048656C70206D6573736167652057
:102D7C00666F722070757A7A6C65203100000000E5
:102D8C000097009300000000009A06E813E005E3AA
:102D9C00050000000066079507E0052F0706070DE4
:102DAC00072007000000000C0FE210FC0B000000D5
:102DBC00007315E81315155315E7140115F31400DA
:00000001FF
